:040000006F008052BB
:100004000000000000000000300300003203000084
:1000140000000000260500000000000000000000B1
:100024002605000026050000000000000000000076
:100034002605000000000000260500000000000066
:100044002605000026050000260500002605000000
:1000540026050000260500002605000026050000F0
:1000640026050000260500002605000026050000E0
:1000740026050000260500002605000026050000D0
:1000840026050000260500002605000026050000C0
:1000940026050000260500002605000026050000B0
:1000A40026050000260500002605000026050000A0
:1000B400D4020000260500002605000026050000E5
:1000C4002605000026050000260500002605000080
:1000D4002605000026050000260500002605000070
:1000E4002605000026050000260500002605000060
:1000F4002605000026050000260500002605000050
:10010400260500002605000000000000260500006A
:1001140026050000000000000000000000000000B0
:1001240000000000000000000000000000000000CB
:0C013400000000000000000000000000BF
:10014000397101436EC619A0397141536AC866CA34
:1001500062CC5ECE19A0397101535AD056D252D416
:100160004ED64AD826DA22DC06DE3301614082828E
:1001700041114AC026C222C406C68282B24D410144
:10018000024D924C224CB24B4101024B924A224A00
:10019000B2494101024992442244B2404101828065
:1001A0003D432A876373C3029377F700BDEFADE544
:1001B000937606FF3D8ABA960CC34CC30CC74CC756
:1001C0004107E36BD7FE11E28280B306C3408A0683
:1001D0009702000096966780A6002307B700A30643
:1001E000B7002306B700A305B7002305B700A30493
:1001F000B7002304B700A303B7002303B700A3028B
:10020000B7002302B700A301B7002301B700A30082
:10021000B7002300B700828093F5F50F9396850011
:10022000D58D93960501D58D61B7939627009702DA
:10023000000096968682E78086FA9680C1171D8F09
:100240003E96E374C3F8A5B7EFF29FF241118545DE
:100250004145EF00F00489677C82C1473EC64C00EF
:100260008D47371501403EC4B126896537150140D9
:100270001121410105B7EFF2BFEFF937112019BF86
:10028000EFF21FEF011185450545EF00500385672B
:10029000938777383ECA4C089D47370500403ECCCF
:1002A000231E0100EF0090030546854537050040F9
:1002B000EF00B00B9307C0027C868D475C87680017
:1002C00085473EC84D2D854537050040EF00700835
:1002D0000561C9B5854537050040EF00300A39C5CD
:1002E00093859181938681819C21982213869181A7
:1002F000850705071377F70F93F7F70F9CA198A2CF
:10030000A54563F7E500238006008546A38DD180CF
:100310001307700C6377F700054723000600238D51
:10032000E180854537050040EF00D006730020309E
:1003300001A0B707EFBE37E700E0938707083CC787
:1003400001A0EFF2FFE205452525252AEF007013F5
:10035000716513050520EF003018313FB707002005
:1003600083A5070837250000130505F4EF001022C8
:100370003D2CAA8537250000130505F5EF00102157
:100380000544B72400001305803EEF00901101CC16
:1003900001460144896537150140F92C138504F69F
:1003A000EF001030CDB705460544EDB7EFF25FDC46
:1003B000371402401C403707FF08411193E717002C
:1003C0001CC05C40F98F5CC01C403707F7FE6D17FE
:1003D000F98F1CC01C403707FCFF7D17F98F1CC02C
:1003E0005C40370701FF7D17F98F5CC0B7079F009E
:1003F0001CC4752E02C402C6B727024023A0070002
:100400001C404167B7160240D98F1CC03706020056
:1004100005679C42F18F3EC6A24785073EC4B2479E
:1004200081E7A247E397E7FEB71702409C43139783
:10043000E7006350070485473EC632478547631C83
:10044000F702B7170240D843B7160240D8C3D843C3
:10045000D8C3D843D8C3D843719BD8C3D8431367F4
:100460001700D8C31147DC42B18BE39EE7FE410180
:1004700015B302C6D9B7372702401C43F19B1CC3F2
:10048000FDB7B7160240DC42370700201146B18B9A
:1004900013070708638FC70221466381C70495EBE2
:1004A0009C42918B9DC7B7470F00938707241CC3BD
:1004B000B7170240DC43918393F6F700B70700209B
:1004C00093870700B69794231C43B3D7D7001CC368
:1004D0008280B7177A0093870720D1BFDC42D442CD
:1004E0004166C983BD8BF18E890745466393C7007A
:1004F000C94781EEB746024083A60680C18A89CEED
:10050000B7167A009386062021A8B7160240D44277
:100510001396E600E35606FEB7163D009386069056
:10052000B387D70269B701A0970100209381813575
:1005300017510020130101AD17250000130505AE6A
:1005400097050020938505AC1386818163FAC50069
:100550008322050023A0550011059105E3EAC5FE9D
:1005600013858181938541846377B500232005003D
:100570001105E36DB5FEFD42739002BC8D42739090
:1005800042809302800873900230970200009382A9
:10059000A2A793E2320073905230EFF03FE197024E
:1005A0000000938242DA739012347300203003A566
:1005B000018282809C4513F7070113F8F70001C7F9
:1005C000D8413368E8008E2113F7F50F39C318417D
:1005D0008146854E3D4F930F800293028004214E49
:1005E0003396DE00B3F8C500631116039398260016
:1005F00033131F011343F3FF3377E300B3181801DC
:1006000033E7E800639FF70550C98506E39AC6FD06
:1006100018C11307F00F6375B70454412146854E86
:100620003D4F930F800293028004414EB398CE0059
:1006300033F715016392E8021317260001173313ED
:10064000EF001343F3FFB376D3003317E800D98EDE
:10065000639DF701232A15010506E319C6FD54C160
:100660008280E39457FA10C94DB7E39757FE2328C9
:100670001501DDB70CC9828019C20CC982804CC932
:100680008280370700C0B377E5006395E708370736
:1006900001405C439356B501584F9D8A9DE6F99BF6
:1006A000B70600FFFD16758F89C993160501C18233
:1006B000D58FB706FF01758D498FB7060007D58F17
:1006C000B7060140DCC2D8CE828005466396C600DC
:1006D000F59BB70680FFF9B709466396C600ED9B08
:1006E000B706E8FFC1B70D466396C600DD9BB706A7
:1006F000FCFF4DBF11466397C60093F7F7F3B706AB
:10070000C0FF4DB71546E391C6FA93F7F7CFB7068A
:10071000E0FF49BF370700406391E702B707014098
:10072000D84F4205B367A70089E51345F5FFB377B6
:10073000E500370701405CCF8280A9E3370801401C
:10074000B70730000326480013170501B376F500FC
:1007500041836396F602B70600F9FD16B377D6001B
:1007600003264800F18E2322D80091C55581120539
:100770003315A700C98F370701405CC382809317E8
:10078000B50063D007029357050193F6F7008D4734
:10079000B397D70093C7F7FFF18FB7060007D58F40
:1007A000E9B7935755019207B317F700E5B7EFF292
:1007B0003F9C37F4FF1F032744723706003E411168
:1007C000931797019346F7FFF18F060737063E0010
:1007D000718FD98F3706000113979600718FD98FCB
:1007E000BD824167F98E02C202C402C6D58F23A220
:1007F000F182035784728545239EE18003270472AA
:100800001305D00323A4E1820327447023A0E182CF
:10081000035704732396E1826124832744703707CA
:100820003A101307077093F7F7F06383E710636AD2
:10083000F7003707321013070770638FE70641018F
:1008400091BA37073B1013070770638BE708370728
:100850003D1013070770E394E7FE854521651535C4
:1008600037140140E177930480044C0013050480A1
:100870007C8226C681338567938787334C001305B6
:1008800004C07C8226C63D3391477C824C0093078E
:100890008002130504C03EC6313BF9774C00371582
:1008A00001407C8226C639338D477C8226C64C00A7
:1008B00013050440013361B7E1773715014093C751
:1008C00007C0130480044C00130505C07C8222C6B7
:1008D000D53189677C8222C64C0037150140D9BFCB
:1008E00085452165793B37140140E1779304800405
:1008F0004C00130504807C8226C66D3993070021C5
:100900004C00130504C07C8226C66D3191477C8261
:100910004C0093078002130504C03EC66139F97785
:100920004C00371501407C8226C669318947B5BF26
:10093000B7140140E17793870770130480044C00DB
:10094000138504807C8222C6B531930790E34C0066
:10095000138504C07C8222C6B13991477C824C0049
:1009600093078002138504C03EC6A931F9779DB76D
:1009700023A8A182828003A70183854714216310E5
:10098000F7021C31639CE7023C21960793E707F8C6
:1009900037E700E093F7F70F36972300F740054756
:1009A00093D756003317D700544189CE9387070455
:1009B0008A07B7E600E0B69798C38280EDF33C2142
:1009C0009607F9B793870706E5B7371702405C43E8
:1009D0009146B18B638CD706A146638ED706BDE7DF
:1009E0001C43918BA5C7B7470F00938707241CC1F1
:1009F000371602405C423707002013070701918336
:100A0000BD8BBA9794231C41B3D7D7005CC1544225
:100A1000A1829D8ABA969422B3D6D70014C55442B7
:100A2000AD829D8A36971423B3D6D70054C5584259
:100A3000634C07005C42B98313F73700938741800A
:100A4000BA979C23B3D7F6021CC98280B7177A00E5
:100A50009387072069BF5C435843C166C983BD8B38
:100A6000758F8907C5466393D700C94701EF37479C
:100A7000024003270780418B09CF37177A001307FD
:100A8000072021A83717024058439316E700E3D602
:100A900006FE37173D0013070790B387E70281BFB3
:100AA00099C5371702401C4F5D8D08CF8280B7175C
:100AB0000240984F1345F5FF798D88CF828099C504
:100AC000371702405C4F5D8D48CF8280B7170240D8
:100AD000D84F1345F5FF798DC8CF82801E21373757
:100AE0000140130707C0C207C1836300E50237074F
:100AF0000040630CE500130707406308E500371763
:100B00000040130707806316E500FA2193F7F7F812
:100B1000D98F9A2593F7F7CFC207C183D98F37179B
:100B200000401EA1130707809C416310E5025CD5BD
:100B3000DE211EB5B7370140938707C06314F50067
:100B4000BC251EB985475EA98280C207C1835EB5F8
:100B5000C5B71E2189C593E717001EA18280C20771
:100B6000C183F99BC207C183CDBF5E2501C6DD8D60
:100B70004EA5828093C5F5FFFD8DDDBF1E294A2558
:100B8000ED8F4205418189C76D8D3335A00082808C
:100B90000145828093C5F5FFC205C1810EA98280FF
:100BA000EFF20FDD1629F577FD17F58FF621DA251F
:100BB0007971D58F1EA95625FD779387379FF58FBD
:100BC000D6212A842EC6D58F9625D58FB625D58FCA
:100BD0005EA55E29C207C18393F7F7CFD98F5EA9BF
:100BE0006808E533B747014093870780B245631A29
:100BF000F404A25756246547B387E702C206C186AC
:100C0000984163D20604060752244206B3D7E7028E
:100C1000130740064186B3D6E702B3F7E702920610
:100C2000635506028E0793872703B3D7E70213F7AE
:100C30007700B367D700C207C1831EA445616FF078
:100C40006FD5925745BF0A07C1B79207938727030D
:100C5000B3D7E702BD8BD58FF9BF91C55E25096774
:100C6000D98F5EA582805A25F977FD17F98FD5BFF8
:100C700093F5F51F4EA182800A216D8D3335A000BA
:100C80008280B707002083A707080967130707F4C6
:100C9000B3D7E702C207C183239BF182239AF18273
:100CA0008280B7F700E0D8438146799BD8C303D749
:100CB00041833306A70290CBD4CB98431367070137
:100CC00098C398431367170298C3D843058B75DF01
:100CD0009843799B98C38280EFF28FC92A8411656B
:100CE0000111854511056D3B930700207C82371566
:100CF00001408D473EC44C00E147130505803EC6C8
:100D0000EFF05F8B22C837440140B70708000C089A
:100D1000130504803ECC02CA231E010051358545CF
:100D2000130504801D3F05616FF0CFC6EFF2AFC21F
:100D3000B7440140AE8932890144938404806345FD
:100D400024014A856FF06FC49305000426852D3772
:100D500065DDB38789008385070026850504C20504
:100D6000C1813937E9BF138781801C439386418451
:100D70003E95636BD500B75600209386068063E5E9
:100D8000A60008C33E858280FD57EDBF39713EDA6B
:100D90002ED232D436D63AD842DC46DE9387C18092
:100DA00022CC804326CA06CEAA8409C41C4C99E3EF
:100DB0002285ED290C4454102686228536C6EF0084
:100DC0007012F2406244D24421618280011126CA2D
:100DD0004AC806CE22CC4EC652C4AA842E8901C56A
:100DE0001C4D91E3E1219C4C804499E326857D29AB
:100DF000971700009387C71A631BF402C0405E2454
:100E0000A18BB1C71C48A1C7FD59294A1C44834581
:100E10000900FD17B1E91CC463DD07062286A94558
:100E200026856120FD576308F502294535A09717EF
:100E300000009387E7186314F4008044C9B797173C
:100E400000009387E713E31CF4FAC0444DBFA2856A
:100E50002685112A55D97D55F2406244D244424933
:100E6000B249224A056182801CC4050963D7070084
:100E7000184C63CAE700638845011C4013871700BC
:100E800018C08CA361B7228626850520E31035F9AA
:100E9000D9B71C401387170018C0294798A371B70A
:100EA0009387C180AA85884315B7011122CC26CA31
:100EB0004AC806CE4EC6AA842E89328401C51C4D6E
:100EC00091E3ED26971700009387870D6317F406CB
:100ED000C0401C4C1CC45E24A18BC1C31C48B5CFB0
:100EE0001C4808409379F90F1379F90F1D8D5C4860
:100EF0006346F500A2852685692C25E51C44050579
:100F0000FD171CC41C401387170018C0238037012D
:100F10005C486388A7005E24858B81CBA947631654
:100F2000F900A2852685B5240DEDF24062444A857C
:100F3000D2444249B24905618280971700009387E5
:100F400027086314F400804469B79717000093875B
:100F50002703E310F4F8C044ADBFA2852685212005
:100F600041D17D59D9B741119387C18026C28443AD
:100F700022C44AC006C62A892E8489C49C4C99E39F
:100F800026852D269717000093878701631BF4029F
:100F9000C0400317C40093170701C18393F687006D
:100FA000ADEA93F6070195EEA5472320F9001367F4
:100FB00007045AA47D55B24022449244024941019B
:100FC0008280971700009387A7FF6314F400804482
:100FD000C9B7971700009387A7FAE31CF4FAC04437
:100FE0004DBF918B9DC34C5889C9930744046384BA
:100FF000F5004A853123232A04025E2423220400BB
:1010000093F7B7FD5EA41C481CC05E2493E78700DD
:101010005EA41C4899EB5E241307002093F7072871
:101020006385E700A2854A85A1215E2413F7170096
:101030001DC35C4823240400B307F0401CCC1C48AB
:101040000145B5FB8317C40013F707082DD793E7B5
:1010500007045EA485B7898B014791E3584818C4FB
:10106000F9BFDE25011122CC26CA06CE4AC84EC6DB
:1010700013F78700AA842E8479EBD841634DE000F2
:10108000B841634AE0000145F2406244D24442491B
:10109000B2490561828058547DD703A90400939614
:1010A000370123A0040063DB060670485E24918BA1
:1010B00099C75C401D8E5C5899C33C401D8E5C54A2
:1010C0000C50814626858297FD575A24631DF500F2
:1010D0009440F54763E8D706B70740208507B3D7A4
:1010E000D700858BA5C31C48232204001CC093177E
:1010F000370163D80700FD576314F5009C4091E366
:1011000068C84C5823A02401BDDD930744046384C0
:10111000F5002685F526232A0402B5B70C500146B2
:10112000854626850297FD572A86E311F5F89C40EF
:10113000B5DF75476385E70059476393E70423A04C
:10114000240191B7136707045AA47D5535BF83A9BD
:101150000501E38A09F203A905008D8B23A035015F
:1011600033093941014791E3D84918C4E35D20F1BF
:101170001C540C50CA864E86268582976347A00071
:101180005E2493E707045EA4C9B7AA993309A9406E
:10119000F1BF9C49B9CF011122CC06CE2A8411C5DA
:1011A0001C4D81E72EC61922B24597170000938780
:1011B00027DF639BF5004C408397C50095C72285C8
:1011C0006244F240056171BD97170000938747DFC5
:1011D0006394F5000C44CDB797170000938747DA66
:1011E000E39CF5FC4C44C9BFF240624401450561F3
:1011F000828001458280411122C406C62A844EA500
:1012000072A52320050023220500232405002322A4
:10121000050623280500232A0500232C0500214666
:1012200081451305C505EFE0BFF7971700009387C9
:1012300047B15CD097170000938767B31CD497170A
:101240000000938747B75CD4971700009387A7B92E
:1012500000D01CD8B2402244410182809705000092
:10126000938565F3A9A2411126C2130680069384D3
:10127000F5FFB384C4024AC02E8922C406C69385F2
:1012800044071D262A8401CD2320050023222501A1
:10129000310508C4138684068145EFE07FF022857E
:1012A000B240224492440249410182801C4DADE388
:1012B000411106C622C497070000938767FA1CD520
:1012C000938701819C4323240504232605042328B6
:1012D00005046314F50085471CCD2A841D2848C0E9
:1012E0002285052808C422852D2048C4484001468F
:1012F0009145113708440546A545F53D4844094642
:10130000C945D53D85471CCCB2402244410182806D
:10131000828041119387018126C284434AC006C658
:101320009C4C22C42A8999E32685493793848404F6
:101330008044DC40FD1763D607009C40B9CF844051
:10134000C5BF0317C40039E7C17785072322040608
:101350002320040023220400232404005CC4232847
:101360000400232A0400232C040021468145130590
:10137000C405EFE0FFE2232A0402232C0402232405
:101380000404232604042285B240224492440249E4
:10139000410182801304840671BF91454A85E1357D
:1013A00088C051FDB1472320F9000144E9BF79719C
:1013B00022D44AD052CC56CA5AC85EC606D626D2C5
:1013C0004ECE2A8AAE8A130485040149054BFD5B83
:1013D00009ECB25022544A8592540259F249624AA9
:1013E000D24A424BB24B4561828004448329440077
:1013F000FD1963D409000040E1BFDE24637BFB00DC
:101400008397E40063877701A6855285829A3369C2
:10141000A90093848406E9BF1971A6DAAE84839586
:10142000E500A2DC86DE328463DB0500DE2423A037
:10143000060093F7070885E7930700401DA03008D2
:1014400036C6EF00D01FB246E34205FE7247BD67C5
:10145000F98F7977BA9793B717009CC2F1BF9307BA
:1014600000041CC0F6506654D654014509618280C0
:10147000DE25011122CC06CE26CA4AC8898B2E84CD
:1014800089CF930774041CC01CC885475CC8F24010
:101490006244D24442490561828074003000AA84CB
:1014A000A53FA2452A892685012219E98317C40090
:1014B00013F7072069FFF19B93E727005EA4D1B7DC
:1014C000970700009387C7D99CD45E2408C008C83A
:1014D00093E707085EA4A2475CC8B24781CF831593
:1014E000E4002685EF00501811C55E24F19B93E7B8
:1014F00017005EA45E243369F9002316240141BF5E
:10150000DDC183A7C5FF411122C406C626C21384CC
:10151000C5FF63D307003E94AA84EF00B01B9387F6
:1015200081839C4381EF2322040023AC81822244E7
:10153000B2402685924441016F00F019637EF400A9
:1015400014403307D4006396E7009843DC43369792
:1015500018C05CC0D9BFBA87D84319C3E37DE4FE85
:1015600094433386D700631F86001040B29694C31D
:101570003386D700E31DC7FA10435843B29694C38D
:10158000D8C375B76375C400B1479CC04DB7104050
:10159000B306C4006316D70014435843B29614C070
:1015A00058C0C0C369B78280011126CA9384350030
:1015B000F19806CE22CC4AC84EC6A104B14763F3C7
:1015C000F404B14463E2B4042A89EF00B0109387B5
:1015D000818398433A8439E09387C1839C4391E7A0
:1015E00081454A85052F23AEA182A6854A851D2700
:1015F000FD5963193507B1472320F9004A85EF00EB
:10160000900D29A0E3D004FCB1471CC10145F24074
:101610006244D2444249B249056182801C40858FB0
:1016200063CF0702AD4663F6F6001CC03E9404C0CB
:1016300031A05C406313870223ACF1824A85EF003E
:1016400090091305B4009307440061993307F540EE
:101650005DDF3A94898F1CC05DBF5CC3C5B722872C
:10166000404095BF130435007198E30285FCB30533
:10167000A4404A854525E31C35FBB5BF1C46FD1734
:101680001CC663DA0700184E63C5E700A9476394D8
:10169000F5006FF09F811C422E851387170018C23A
:1016A0008CA38280011122CC26CA4AC84EC652C4DD
:1016B00006CE2A89AE893284B304D6007D5A6314DB
:1016C0009400014501A80C204E864A85453F05043B
:1016D000E31745FFF2406244D2444249B249224AEC
:1016E00005618280357122CD26CB4AC94EC706CF0F
:1016F00052C556C35AC1DEDEE2DCE6DAAA89AE8400
:101700003289368401C51C4D91E34D369717000090
:10171000938707896397F40C83A44900DE24A18B87
:10172000FDC39C48EDC393070002A304F102930795
:10173000000302D22305F10222C6930B5002971A2E
:101740000000938AEA89054C294B4A841C2099C3DE
:10175000639E770DB30C2441638D0C00E6864A86A8
:10176000A6854E858137FD57630FF51C9256E69688
:1017700036D21C206389071CFD571309140002C8C8
:1017800002CE3ECA02CCA309010482D483450900DB
:1017900015465685252713041900C24751E913F74A
:1017A000070109C713070002A309E10413F7870023
:1017B00009C71307B002A309E10483460900130710
:1017C000A002638FE606F2474A8481462546182028
:1017D00093051400130707FD6377E60AB5CA3ECEEA
:1017E00085A8970700009387A77D6395F40083A4DD
:1017F00089002DB79707000093878778E390F4F26C
:1018000083A4C90021BFA6854E85EFF0CFF501DD89
:101810007D55FA406A44DA444A49BA492A4A9A4A02
:101820000A4BF65B665CD65C0D618280050439BFAD
:10183000330555413315AC00C98F3EC82289B9B76D
:10184000324793064700184336C6634707023ACE2D
:1018500018209307E002631DF70418309307A002D5
:10186000631BF702B2470904138747009C433AC63B
:1018700063C107023ECA2DA83307E04093E7270063
:101880003ACE3EC8F1B7B387670385462E84BA9730
:101890003DBFFD57C5B7050402CA814681472546AD
:1018A000182093051400130707FD6374E606F9F288
:1018B0000C200D461705000013050573012511CDF9
:1018C00097070000938747721D8D93070004B39715
:1018D000A700424505045D8D2AC80C20194617054E
:1018E00000001305A570130914002304B102F923A5
:1018F00035C197E7FFFF9387E77095E74247B24707
:101900001377071009CF91073EC69257D2973ED260
:101910002DBDB387670385462E84BA9751B79D07BF
:10192000E19BA107D5B77800970600009386C6D73C
:1019300026860C084E8597000000E7000000FD5742
:101940002A8AE314F5FCDE2493F70704E39207ECFC
:101950001255C1B57800970600009386E6D4268616
:101960000C084E85012AE1BF797156CA9C49BA8A92
:10197000984522D426D24ECE52CC06D64AD05AC84A
:101980005EC6AA892E84B284368A63D3E700BA87FA
:101990009CC00347340419C385079CC01C4093F7BF
:1019A000070281C79C4089079CC003290400137962
:1019B0006900631A0900130B9401FD5B5C449840B5
:1019C000998F634CF9041C408346340493F7070253
:1019D000B336D000A5EB13063404D2854E85829A27
:1019E000FD576303F5041C4011469840998B5444FD
:1019F00081446397C700B384E64063D30400814405
:101A00001C4418486354F700998FBE940149690437
:101A10007D5B63982405014509A885465A86D285D1
:101A20004E85829A631E75017D55B25022549254A0
:101A30000259F249624AD24A424BB24B4561828016
:101A40000509ADBF3307D40013060003A301C70483
:101A50000347540493871600A2978906A381E704DD
:101A60009DBF85462286D2854E85829AE30E65FB10
:101A7000050945B7797122D426D24AD04ECE06D672
:101A800052CC56CA5AC8B689942D9307900632890B
:101A9000AA842E8413863504638DF60263E2D7068A
:101AA000930780056385F61863EDD700638D0620E4
:101AB00093073004638EF60A930A24042301D404A6
:101AC000C9A0930730066385F60A93074006E3959D
:101AD000F6FE1C40084393F6070893054500C5C66B
:101AE0001C410CC363D807001307D002B307F040B2
:101AF000A301E404970600009386C64F294765A812
:101B0000930700076381F61663E5D7029307E006A3
:101B10006388F6189307F006E390F6FA0C401C432E
:101B200013F80508138547006307080608C39C439C
:101B300085A893075007E383F6FE93078007638821
:101B4000F61293073007E399F6F61C43D04181451E
:101B50009386470014C383AA07005685852601C5CE
:101B60003305554148C05C401CC8A301040461A86A
:101B70001C43930A2404938647009C4314C3230107
:101B8000F4048547D5B793F607041C410CC3B9DAB2
:101B9000C207C18781BF93F5050408C3C9D99E2335
:101BA0001307F0066386E60E9706000093868644C8
:101BB0002947A30104044C400CC463C50500084038
:101BC0006D9908C099E3B28A89CDB28AB3F5E7026C
:101BD000FD1AB6958C212380BA00B3D5E70263FFC6
:101BE000E70AA147631EF7001C40858B91CB584044
:101BF0001C4863C7E70093070003A38FFAFEFD1A92
:101C00003306564110C84E87CA867000A2852685C5
:101C1000A13B7D5A631D450B7D55B2502254925411
:101C20000259F249624AD24A424B45618280A382FC
:101C3000D504970600009386E63B0C40084313F852
:101C400005081C411105630D080208C313F71500B0
:101C500001C793E505020CC04147A1FF0C4093F575
:101C6000F5FD0CC0B9B79C4193E707029CC19307EF
:101C70008007A302F404970600009386E63875BF38
:101C800013F8050408C3E30308FCC207C1837DBF42
:101C90009706000093860636214721BFAE873DB7E1
:101CA00094411C43CC4913F806081385470063068A
:101CB000080008C39C438CC339A008C393F60604EC
:101CC0009C43F5DA8EA323280400B28A2DBF144862
:101CD0005686CA8526858299E30045F51C40898B86
:101CE0008DE7B2474844E35AF5F23E853DB7854655
:101CF0005686CA8526858299E30065F3050A5C4409
:101D00003247998FE345FAFEE9BF014A930A9401ED
:101D10007D5BF5B7411122C42A842E8523A001845E
:101D200006C6EFF04F84FD576317F50093870184D3
:101D30009C4391C31CC0B2402244410182804111A6
:101D400022C42E848395E50006C6792263490500E6
:101D50007C48AA977CC8B2402244410182805E241C
:101D60007D777D17F98F5EA4FDB7DE25011122CCAA
:101D700026CA4AC84EC606CE93F70710AA842E84F8
:101D80003289B68991C78395E500894601460922C3
:101D90005E247D777D17F98F5EA48315E40062448D
:101DA000F240CE864A86B24942492685D244056130
:101DB00025A8411122C42E848395E50006C6C928B2
:101DC000FD575A24631AF500FD77FD17F98F5EA4BD
:101DD000B2402244410182808567D98F5EA468C8E1
:101DE000C5BF8395E50005A8411122C42A842E852C
:101DF000B285368623A0018406C6EFE03FF3FD5787
:101E00006317F500938701849C4391C31CC0B240C3
:101E1000224441018280411122C42A842E8523A0BC
:101E2000018406C6C520FD576317F500938701841A
:101E30009C4391C31CC0B2402244410182804111A5
:101E400022C42A842E85B28523A0018406C6C92017
:101E5000FD576317F500938701849C4391C31CC011
:101E6000B240224441018280411122C42A842E853D
:101E700023A0018406C65D20FD576317F5009387F4
:101E800001849C4391C31CC0B24022444101828022
:101E9000411122C42A842E85B285368623A001846E
:101EA00006C65920FD576317F500938701849C43AC
:101EB00091C31CC0B24022444101828093F5F50FCA
:101EC0002A966314C500014582801C21E38EB7FE6B
:101ED0000505C5BF82808280411122C42A842E85D7
:101EE000B285368623A0018406C6A920FD57631754
:101EF000F500938701849C4391C31CC0B2402244E7
:101F0000410182809307800523A0F1847D55828062
:101F10009307800523A0F1847D5582809307800577
:101F200023A0F184014582809307800523A0F184DA
:101F30007D5582809307800523A0F1847D558280A2
:101F400053797374656D436C6B3A25640D0A000018
:101F50004368697049443A253038780D0A0000001A
:101F600054686973206973207072696E74662065A5
:101F700078616D706C652063630D000000000000E7
:101F80000000000000000000000000000000000051
:101F90000000000000000000000000000000000041
:101FA0000000000000000000000000000000000031
:101FB0000000000000000000000000000000000021
:101FC0000000000000000000000000000000000011
:101FD000000000000000000000000000232D302B56
:101FE00020000000686C4C006566674546470000AD
:101FF000303132333435363738394142434445463F
:102000000000000030313233343536373839616200
:08201000636465660000000036
:102018000000000000000000010203040607080990
:102028000000000001020304010203040607080976
:10203800000000009C1F0000BC1F00007C1F000067
:102048000000000000000000000000000000000088
:102058000000000000000000000000000000000078
:102068000000000000000000000000000000000068
:102078000000000000000000000000000000000058
:102088000000000000000000000000000000000048
:1020980000127A0002040608C40000202000002074
:0820A8002000002000000000F0
:00000001FF
